:030000000219FDE5
:03000B000200AA46
:03002B0002015679
:03005B000202ECB2
:030073000202D2B4
:1000800002030406080C10182030406080040608A3
:100090000C10182030406080A0C000070F1F3F0DDB
:1000A0000D0403060D0503030202C2AFC0D0C0E079
:1000B000206217E5256002E473E525F4F58A758B67
:1000C00000D262D0E0D0D0D2AF3285268AC262E5BB
:1000D00026F46035306803207210758B00D0E0D0B4
:1000E000D0D295D293D297D2AF32D295D293D29723
:1000F000206E0C206609740CD5E0FDE57E429075FB
:100100008B00D0E0D0D0D2AF32758A00C28DD262DF
:1001100001FF01B9306805206602C29501B9306857
:1001200005206602C29701B9306805206602C293B5
:1001300001B9C294306805206602C29501B9C29621
:10014000306805206602C29701B9C2923068052066
:100150006602C29301B9C2AFC2AD53E6EFC0D0C0D0
:10016000E0D2D3D2AFC2CEE52A6007207449152A67
:1001700021B77800790020742EE580307E01F430BC
:10018000E50278FF53DACF207E0343DA20307E0386
:1001900043DA10C2D8C271E580307E01F430E50246
:1001A00079FFC3E89970CB306103752A402074034E
:1001B000752A40885FD27020740DE52B6004152BE2
:1001C00021C743DA01C2D820700221DAA85F20617A
:1001D00002C27020740221D888227882B604038576
:1001E0002224C3E52594404002D26420CF0AD0E007
:1001F000D0D043E610D2AD32C2CF053A7802E52A1C
:100200006005307402152AC3E55F940140057562EC
:10021000004124756300756C00E5622401F56250AD
:10022000037562FF7982B7020D306D1DC3E522941C
:10023000324016854D227982B7030E306D0BC3E52F
:100240002294324004798E8722C3E52395226008E8
:100250004004152341580523D8CA056CE56C70028B
:10026000156CD56D63756D017805C3E56C956E40B1
:1002700057C3E56C956F50087801756D0302028CC9
:10028000C3E56C957050057801756D01C3E5659502
:1002900024401E7982B7040241BD206D1485246577
:1002A000E56C046003856E6C756D0175233C02027C
:1002B000C8E5652850057565FF41BDF565E5650430
:1002C00070067563FF756CFFD0E0D0D043E610D2A6
:1002D000AD32C2AFC0D053E67FC260759100855683
:1002E00094855795759104D0D0D2AF32C2AF53E602
:1002F000EFC2ADC0D0C0E0C0F0D2D3D2AFA8FBA94E
:10030000FCC2D8307102615353DACF207E0343DA46
:1003100010307E0343DA20D271E580307E01F42074
:10032000E502612A88278928A13253DACF207E038B
:1003300043DA20307E0343DA10C2D8C2713074022F
:10034000A11E7800E580307E01F430E502A11E8810
:100350005FA10653DACF207E0343DA20307E0343C9
:10036000DA10C271206102812C53DACF207E034360
:10037000DA10307E0343DA20C2D8D271885A895B02
:10038000C3E89558F8E99559F97B007E087A00C3CF
:10039000E8948CE994005005755E00811E882178F0
:1003A000A2E6A8216055C3E894C8E994005008E487
:1003B000D2E4FB7A0A61F9C3E89468E99401500831
:1003C000E4D2E3FB7A0F61F9C3E894D0E9940250D8
:1003D00008E4D2E2FB7A1E61F9C3E894A0E994052F
:1003E0005008E4D2E1FB7A3C61F9C3E89498E994BF
:1003F000085008E4D2E0FB7A787E00C3E8955CFC04
:10040000E9955DFD30E70AECF42401FCEDF43400DD
:10041000FD755E00C3EC9AED9E5003755E01885C2D
:10042000895D855A58855B597802A106C3E89527EE
:10043000F8E99528F9307C0281EA307B0281EA30C4
:100440007A0281E3207502814FE9FDE8FC816EE9C3
:10045000C313F9E813F830790281E3E9C313F9E82B
:1004600013F830780281E3E9C313FDE813FC20613F
:0F04700026C3EC941CED940240028185ED7018B8
:10047F00C3EC94C850120529C3E529940A5002A170
:10048F001E755F00D270A11EE52960021529740048
:10049F00207F037896E624FAFEE43400FFC3EC9E37
:1004AF00FCED9FFD50067800790081EAC3EC94FFC4
:1004BF00ED9400400678FF790081EAEC8575F0A491
:1004CF00C5F0A2F733F87900400302050678FF79EB
:1004DF0000020506E9C313F9E813F8307C0EE96052
:1004EF000278FFC3E81338F8E43400F9C3E894FF47
:1004FF00E99400400278FF885FD270206102A11E4C
:10050F00741FF4552F4BF52FC274EB7002D2747514
:10051F002A40307403752A0A306102A13220740315
:10052F0053DAFE207403752B20D0F0D0E0D0D0D258
:10053F00AD43E61032790102056279030205627953
:10054F000A020562791E020562796402056279C8A2
:10055F000205627817E4D5E0FDD8FAD9F6227A14AD
:10056F007B780205897A107B8C0205897A0D7BB422
:10057F000205897A0B7BC80205897902B27DE4C234
:10058F0096D5E0FDC297D5E0FDD297D5E0FDD29686
:10059F00D5E0FDC295E576D5E0FDD2957496D5E010
:1005AF00FDD9D9EAF8D5E0FDD8FBDBCEC29622C340
:1005BF007C007D0075F00005F0EA33FAEB33FB5059
:1005CF00F6EB13FBEA13FAC3E9FFE8FEE89AF8E942
:1005DF009BF95004EFF9EEF8B3EC33FCED33FDD596
:1005EF00F0DFEDF9ECF822E889F08A20D2D4F8A9EF
:1005FF00F07B0030F70B7BFFF42401F8E9F43400B3
:10060F00F9E88520F0A4ADF0F8E98520F0A4AFF06B
:10061F00FEED2EF974003FFA7C04C3EA13FAE913D6
:10062F00F9E813F8DCF48BF030F70AE8F42401F85A
:10063F00E9F43400F9E889F0C2D4F8A9F0227882FD
:10064F00B604030206ECC3E55F9419401EE52D5472
:10065F00067018206D3678057994E7146007780ACC
:10066F001460027812C3E54198401F306D09856709
:10067F0065756CFF756D01852224E4F545F546F52A
:10068F0047F548F549C26D0206ECD26D7994E7142F
:10069F007013E523F43333F913F8E9540104F9E83F
:1006AF0054FE0206E0E714147014E523F4333333D9
:1006BF00F913F8E9540304F9E854FC0206E8E523BA
:1006CF00F433333333F913F8E954070404F9E854D6
:1006DF00F8C39440F8E99400F98845894622C3E5A8
:1006EF004113F9E54013F8C3E54598F8E54699F944
:1006FF00500CC3E89480E994FF4016020724C3E826
:10070F00947FE994005003020724787F7900020751
:10071F0024788079FF884A894B22E54A2547F8E5F6
:10072F004B3548F9854B20E4300701F43549FA3051
:10073F00E709C3EA94F04015020762C3EA940F5029
:10074F000302076278FF79FF7A0F02076278007958
:10075F00007AF0C3E5249564500AC37401952450C0
:10076F000B020780E54B20E70E020780E54B30E7D1
:10077F0006884789488A492278A4E6FAC3E54A33AE
:10078F00F8E54B33F9B1F6E930E70BC3E89480E9AC
:10079F0094FF4013E1BAC3E8947FE994005002E15B
:1007AF00BA787F7900E1BA788079FFE820E715C33E
:1007BF00E52398F84009C3E8940140030207E17864
:1007CF00010207E1E8F424012523F840030207E1C1
:1007DF0078FF884C2278A5E6FAA848A949B1F6E92E
:1007EF0030E70CC3E89401E994FF4016020815C3E3
:1007FF00E894FFE99400500302081578FF7900028E
:10080F000815780179FFE920E715C3E54C98F84002
:10081F0009C3E89401400302083C780102083CE850
:10082F00F42401254CF8400302083C78FF88242269
:10083F0078FFC26420693D206A12D264C3E54194F7
:10084F000A4009C3E52594405002C26479A1E760CC
:10085F0023E541601F74FF8541F0848539F0306ACC
:0E086F000375F005A4F8C5F0600278FFC3E839
:10087D0095675002A867886622C3E5409440E5411C
:10088D009401E5665003140197046002F566227821
:10089D0083E6F520120F3575E89012054475E89042
:1008AD00E5E820ECFBA8BDA9BE120FCF75715575FB
:1008BD007200C3740013FD7455606613FC74552CDF
:1008CD00FC74003DFDECFAEDFBC3E89AE99B401486
:1008DD00E5712455F571E5723400F572EA2CFAEBE9
:1008ED003DFB80E5AE71AF72C3E57213F9E571138F
:1008FD00F8C3E913F9E813F87A03C3E913F9E81318
:10090D00F8DAF7AA201A70097571007572000209DC
:10091D002E1AEA6008EE28FEEF39FFDAF88E718F95
:10092D00722275E890227883E6FFE5E820ECF7A8BF
:10093D00BDA9BE0573C3E57394084052757300E9F4
:10094D00FA79A0E76044EA7007E574601B02096953
:10095D00C3E895746010E5745006600C14020975B7
:10096D000460F9020975E574F574C3946D401B7547
:10097D0064C0C394044013756480C39404400B7524
:10098D006440C39404400375640075BB0822EFC333
:10099D009401601F7455601BC3E894FFE9940350E4
:1009AD0012C3E89571E995725009E564600C156400
:1009BD000209C7E564F460020564A864C3E52498E0
:1009CD005002A824C3E89565400AA865E565F46062
:1009DD000385656488258826E573B4070375BB1008
:1009ED0022743279A687F0A4C5F0A2F733F8C3E8D4
:1009FD0095644002A8648822882488258826886703
:100A0D00227540007541F022C2AF75C820A8CCA94F
:100A1D00CDAA3A30CF010A75C824D2AFAB3BAC3C5E
:100A2D00883B893CC3E89BF8E99C206908F930674D
:100A3D0002612A4187AD3D8A3DF9EA9DFA6004784D
:100A4D00FF79FFAE3EAF3F8B3E8C3FC3EC9FFCC3A7
:100A5D00E99CF542A83BA93CC3E89EF8E99FF9C380
:100A6D00E54113FBE54013FAE82AF540E93BF54172
:100A7D0050067540FF7541FF41D1AA40AB41AC40D6
:100A8D00AD417E047F02C3EB940440021E1FC3EBF5
:100A9D00940840021E1FC3ED13FDEC13FCDEF7C3DB
:100AAD00EA9CFAEB9DFBEF6009C3E913F9E813F833
:100ABD00DFF7EA28FAEB39FB8A408B4150067BFFC2
:100ACD008B408B41C3EB94025002D2673069047F97
:100ADD000341FC7892E6FFC3E537948240110FC3C2
:100AED00E53794A040010FC3EF940640027F057EC9
:100AFD0005E541C4540FF9E541C454F0F8E540C48F
:100B0D00540F28F8C3E89EFAE99400FB4009C3EAA4
:100B1D009402EB940050047A02E4FB6176AA40AB98
:100B2D0041EBC4FEEAC4540F4EFCC3EA9CFAEB94AD
:100B3D0000FBC3E813C313F8EA28FAEB3400FB8A71
:100B4D00408B41C3EB94024002C2677805EBC4FEB3
:100B5D007B00EAC4540F4EFAC3EA98FA4005C394D9
:100B6D000250027A027892E6FF3060026176855279
:100B7D0056855357D26043E680C3E49AF8E49BF957
:100B8D003067028110E8FAE9FBD3E913FDE813FCA5
:100B9D0088528953C3EF94036038EF20E00DE82CA1
:100BAD00F8E93DF9ECFAEDFB020BCBE828F8E93951
:100BBD00F9C3E82402F8E93400F97AFE7BFFC3EFAC
:100BCD009403400E8A548B55884E894F8C508D510D
:100BDD008144885489558A4E8B4F8C508D51306984
:100BED0020C3E53394034019E542A2E713F8E55518
:100BFD00F4240138400B20E7087554FFF42401F567
:100C0D00558144E8FAD3E813FC8852C3EF9403608E
:100C1D0020EF20E007E82CF8ECFA8130E8282402D8
:100C2D00F87AFEC3EF940340088A54884E8C5081A5
:100C3D004488548A4E8C50E56BC3335002646BF577
:100C4D006B306002814E753402D26043E680E52D33
:100C5D0054066026A840A941C3E913F9E813F8C268
:0E0C6D00AF53E67F759100C3E498F594E499C7
:100C7B00F595759104D26043E680D2AF22D26575AB
:100C8B004400752000306B03752040020CA7D26521
:100C9B00754400752040306B03752000D2AF78018E
:100CAB00206722E52D54066002C265C3E541940519
:100CBB0040137802940540087803940540027806A7
:100CCB00306902780A206019E544601530690AC35F
:100CDB00E53394034003D53406D2AFD26CA178919F
:100CEB0056D2AF0000C2AF206726E541C3FB940F7D
:100CFB0040027B0FEB240530730123306A0274280A
:100D0B0020620123F93069027982E58BC39940B5E2
:100D1B000544E59B5440B52002A16230690A08C323
:100D2B00E8940A40010881D020650281A7C265536F
:100D3B00E67F7591003067107594007595FE75917F
:100D4B0004D26043E68081A7AE40AF41C3E49EF579
:100D5B0094E49FF595A149C3E5339402500281A712
:100D6B0030650281A7D802A17681D0C26C53E67F91
:100D7B00759100855494855595759104854E5685CE
:100D8B004F57D26043E680D2AFE52D540660082062
:100D9B006A020533020DB2306C0D206B0A20650719
:100DAB001581158102160722780030640530650223
:100DBB007801E53775F007A4F9E5F028F5F0E9A21D
:100DCB00F013A2F113A2F213F537C3947850037505
:100DDB003778C3E53795384008D266D295D293D28F
:100DEB0097306002A1EC855056855157D26043E68F
:100DFB008022207D11C2AF754302C296D294D2AF2E
:100E0B00759F11020FCCC2AF754302C296D292D21C
:100E1B00AF759F11020FCC307243207D20C2AF758E
:100E2B00430390013E757E40D293C292306204C25E
:100E3B0097C140D296D2AF759F13020FCCC2AF753C
:100E4B00430390013E757E40D295C294306204C23A
:100E5B0097C160D296D2AF759F10020FCC207D1731
:100E6B00C2AF75430390011ED293306202C297D278
:100E7B00AF759F13020FCCC2AF75430390011ED207
:100E8B0095306202C297D2AF759F10020FCC207DB6
:100E9B0011C2AF754304C294D292D2AF759F1002A8
:100EAB000FCCC2AF754304C292D294D2AF759F13CD
:100EBB00020FCC307243207D20C2AF7543059001E9
:100ECB0032757E10D297C296306204C295C1DCD2C5
:100EDB0094D2AF759F11020FCCC2AF754305900131
:100EEB004A757E04D297C296306204C293C1FCD27B
:100EFB0092D2AF759F11020FCC207D17C2AF7543F5
:100F0B0005900114D297306202C295D2AF759F1132
:100F1B00020FCCC2AF754305900128D2973062EB1C
:100F2B00C293D2AF759F11020FCC207D11C2AF754A
:100F3B004306C292D296D2AF759F13020FCCC2AFAB
:100F4B00754306C294D296D2AF759F10020FCC3068
:100F5B007242207D20C2AF75430190014A757E0419
:100F6B00D295C294306204C293E178D292D2AF751B
:100F7B009F10020FCCC2AF754301900132757E10EA
:100F8B00D293C292306204C295E198D294D2AF75DB
:100F9B009F13E1CC207D16C2AF754301900128D27F
:100FAB0095306202C293D2AF759F10E1CCC2AF7580
:100FBB004301900114D293306202C295D2AF759F58
:100FCB0013C26622900112757E00D295D293D297EE
:100FDB00C294C292C296C2622278807607087607C4
:100FEB000876010876040876FF0876FF08760A086B
:100FFB007602087601087601788C7601087600086F
:10100B0076B40876FF0876FF0876FF087603087635
:10101B00FF0876010876FF0876250876D0087678E3
:10102B000876C80876040876FF087601087600086B
:10103B00767A08760A087601087601087600087633
:10104B00FF227887E6FFC272BF0302D2727888C292
:10105B007DE630E102D27DC27E7889E630E102D2B4
:0F106B007EC3EF94026008758E01D27302107F6E
:10107A00758E00C273227880E6149000809378A45B
:10108A00F67881E6149000809378A5F67886E614BF
:10109A0090008D9378A6F6789FE6F8700108C3E869
:1010AA00941140027811E82828F56E256E256E28DD
:1010BA00F56F256E2828F570789CE67538FF753926
:1010CA000CB402067538A075390AB403067538825D
:1010DA0075390578A3E61490009A93F569120FCF33
:1010EA0022227896E6FA7897E6FB7888E6B4030532
:1010FA00C3EB940EFB307F047A007BFFC3EB9AFCB0
:10110A00C3948250027C827575000575EC8575F072
:10111A00A4C3E5F0947D40F222D27F11EC1205536C
:10112A007A007B007C10120549E55F2AFA74003BBD
:10113A00FBDCF37C04C3EB13FBEA13FADCF7FEC215
:10114A007F11EC22E5EF20E6037520000520903F91
:10115A00FFE520146006901DFF14600093046003ED
:10116A0075EF1253D9BF7581C043FF8012054475CC
:10117A00EF0243B203E5B3240420E70DF521E5E3CA
:10118A0020E0068521B343E301120FCF7580FF7576
:10119A00A40075F1B275D4DF7590A975A5FC75F236
:1011AA00FE75D50175A60175E241E4F8F6D8FD751C
:1011BA006B01120FE412164F78988676753001C2C9
:1011CA00AF12055D12056D1205531205741205530F
:1011DA0012057B12055312177212055D12055D1274
:1011EA000558C2AF78FA79FA308507D9FBD8F702E1
:1011FA001C00114D118011EB11EC78988676120FB4
:10120A00CF75885075891275C82475910475D840B0
:10121A0075A82275B80275E690759B80759D007554
:10122A00D10E75BC5875BB0875BA1175E8801205E0
:10123A0044D2AF12089C53DACF207E0343DA20301F
:10124A007E0343DA1043DA01C2D8C27112055DD2B5
:10125A00617B037A0CE55E70077A0CDB030211EC02
:10126A001205532070030211ECC270E55FC39402A9
:10127A0040E1E52F541F856160F561B560D5DAD587
:10128A00C26153DACF207E0343DA20307E0343DA89
:10129A0010C2D8C27178A2E67008D274E52F54E061
:1012AA00F52FC275752900120558307409C3E5294E
:1012BA00940A4002D2751205497802307402780005
:1012CA00C3E55F9840F0C2AF12056D12056D1205B5
:1012DA006DD2AF12055D754D00120549788CE6C3D3
:1012EA00940150030213B9E530C394015003021369
:1012FA00B9207435C3E55F94FF50030213B9C2AF36
:10130A00120582D2AF120558C3E55F940150EFC2AD
:10131A00AF12056D12054E12056DD2AF120558C3F4
:10132A00E55F94FF40E90217F77F05D27F11EC12BF
:10133A000558C2AFC27F11ECAE5FC3E55F947FD29E
:10134A00AF4076120544C2AF120582D2AFDFDC315C
:10135A0023C3EE94057897F612055D1216911217BB
:10136A007A7F0AD27F11EC120558C2AFC27F11EC04
:10137A00AE5FC3E55F947FD2AF50E6120544C2AFB9
:10138A0012056D12054E12056DD2AFDFD63123EE6E
:10139A0024057896F612055D1216911217A9120500
:1013AA005811ECC3E55F94FF500241FB0217F7C3E3
:1013BA00E55F954D4003855F4D12055878017988A0
:1013CA00E7B403027805C3E55F98400241E3C2AF80
:1013DA00120582120582120582D2AF12055D75309E
:1013EA0000E4F531F5320531E531F470390532782A
:1013FA009AE67819146012783214600D787D1460B8
:10140A000878FA146003753200C3E532984017155C
:10141A00327531B478998676C2AF120582D2AF7826
:10142A0098867612055812054EE52A700530740220
:10143A0021EC78012074027806C3E55F9840A71270
:10144A000558E52A70030211ECC2AF120FCFE4F57A
:10145A0022F523F524F525F526F56AD2AF7885E637
:0F146A00C333F568E4F545F546F547F548F54910
:10147900F573F52CF52DF53775730875BB10120545
:101489004412092FE5E820ECFBA8BDA9BEE97001CB
:10149900F8887412093375730875BB107887E6FEEE
:1014A9007602114D7887EEF6C2AF7564FF1209EE28
:1014B900852264852265852266D2AF75220175244D
:1014C9000175250175260185636C756D017888E6BE
:1014D900B40307C27D307602D27DD268D2697533F2
:1014E90000120F35120F5A120A0E120A15120A0E9D
:1014F900120A15120A0E02150EC2AF114DD2AF759E
:10150900730075BB08120C9912064D120DB3120D1A
:10151900FD120A15120C88306D031206ED206703BF
:1015290012083F306703120886120DB3120E2212F9
:101539000A15120C99306D03120729120DB3120EF8
:1015490099120A15120C88306D03120787120DB310
:10155900120EBE120A15120C99306D031207E4120D
:101569000DB3120F35120A1512092F120C88120D1C
:10157900B3120F5A120933120A1530692F206B2C36
:1015890085676485676585636C756D0179187A0C63
:10159900C3E533994009C269D26A8A350215B5C3D0
:1015A900E55F9401400302150E02160F306A1B20F5
:1015B9006B18E535147004C26AA102F535C3E55FFD
:1015C9009401400302150E02160F753600C3E56239
:1015D9009401400985676585636C756D01C3E56292
:1015E90078FA985021307404E52A601A78F0306B43
:1015F900058567647820C3E541985002A10E053638
:10160900E55F6002C112753600C2AF120FCF78874D
:10161900E6FE7602114D7887EEF6E4F522F523F51C
:1016290024F525F526F568C268D2AF120544120FD4
:10163900CF307406E52A700221EC788DE6C3940157
:10164900400241C061EB901A0D78201216D3E520B3
:10165900B4A50CA31216D3E520B45A0302167112CD
:101669000FE4121691021690901A0378807B0A12E1
:1016790016D3A308DBF9901A0F788C7B181216D3AE
:10168900A308DBF9901A2722C2AF1217121216EC1F
:10169900901A00740E1216D8A374041216D8A374E3
:1016A900141216D8901A0378807B0A1216D7A30849
:1016B900DBF9901A0F788C7B181216D7A308DBF97F
:1016C900121725121703901A2722E493F622E643EC
:1016D9008F01538FFD75EF0275B7A575B7F1F053FB
:1016E9008FFE22438F02438F0175EF0275B7A575EF
:1016F900B7F1901A0DF0538FFC22901A0D74A5D1F1
:10170900D8901A0E745AD1D8227A3079D07820908C
:101719001A40D1D3E520F709A3DAF7227A3079D034
:10172900901A40E7D1D809A3DAF922AB77A878BB98
:1017390001027980BB02027981BB03027982BB0471
:10174900027994BB05027983BB06027986BB07023D
:101759007992BB08027987BB0902799CBB0A027995
:1017690088BB0B027989E8F7227C0512055DDCFB51
:1017790022C2AF12056D12057412057B1205821281
:10178900054E12056D12057412057B1205821205AC
:101799004E12056D12057412057B120582D2AF2215
:1017A900C2AF12058212057B12057412056D12056E
:1017B9004E12058212057B12057412056D12054E33
:1017C90012058212057B12057412056DD2AF22AE85
:1017D90077AF78C2AF12056D12056D12056D12054E
:1017E9004EDEF212058212054EDFF8D2AF22F17AEF
:1017F900F172F1727577017578017579001217D850
:101809007C05AD5F12055DC3ED955F70F5C3E55FBE
:101819009401400AC3E55F94FF4037021838121754
:101829003412169112177AC2AF75EF12121772DCC1
:10183900D10579C3E5799403500280C11217720565
:1018490078E5771490009F93F808C3E578985002DB
:1018590080A81217721217720577C3E577940C5096
:0E186900028094120FE4121691C2AF75EF12B6
:03187700121772D3
:0319FD0002114E86
:101A00000E041407070104FFFF0A020101A55A0191
:101A100000B4FFFFFF03FF01FF25D078C804FF01DA
:081A200000FF0A010100FFFFB5
:101A400023526F746F724765656B73323041232088
:101A500023424C48454C4923463333302320202031
:101A60002020202020202020202020202020202076
:101C0000C2AFC2D353D9BF7581C043B20343FF8073
:101C1000752438752503B1C975EF0275E24043F1AB
:101C20002053A4DF75D400D2857DFA780379E67C51
:101C300010752200752300901DD67B0675249875BB
:101C400025013085028142208508D8FBD9F9DCF7CF
:101C500081B4308508D8FBD9F9DCF781B4B189E4C7
:101C600093A3C39A6004DDC381B4DBDBB17B600264
:101C7000812B7B08E493FAA3B15CDBF87A30B15C8A
:101C8000752200752300B17BEAFCEBFDC3ED94FEE9
:101C9000400EB17B8A278B28ED30E0048A828B834B
:101CA000B17B7AC270D8C3ED94FE601350CEBD00F4
:101CB00025EC60097520007521FF0200008100A855
:101CC00027A9280809D804D90281D3B17FEA89AAB3
:101CD000F281C50D81A0C3ED94035049EDA2E092BD
:101CE000007AC5C3E5829400E583941C50902000DF
:101CF00010438F02438F0175B7A575B7F1F030001F
:101D00001FA827A9280809438F01538FFDD804D99C
:101D100002A12089AAE275B7A575B7F1F0A3A10DBC
:101D2000538FFC817C7AC1BD030CE493A3FAB140CC
:101D3000DCF8B138817C817EAA22AB23B15CEBFA5E
:101D4000EA6222752608C3E52313F523E52213F57D
:101D50002250066323A0632201D526EAB1C9B1C986
:101D600075260AEAF4200102D285300102C285B14B
:101D7000C9C3134002C201D526EB22B17FEAFB2082
:101D80008502A17F308502A184752608AE24AF2587
:101D9000C3EF13FFEE13FEB1CDB1C9C3EA13308513
:101DA000024480FA30E703632201C3E52313F523DD
:101DB000E52213F52250066323A0632201D526D91C
:101DC000E52265236523F52222AE24AF250E0FDE22
:101DD000FEDFFCD20122424C48656C693437316326
:041DE000F3300601D5
:00000001FF
